:100000000C9469000C9486000C9486000C94860075
:100010000C9486000C9486000C9486000C94860048
:100020000C9486000C9486000C9486000C94E103DA
:100030000C9409040C9486000C9486000C948600A1
:100040000C9486000C9486000C9486000C94860018
:100050000C9486000C9486000C9486000C94860008
:100060000C9486000C9486000C9486000C948600F8
:100070000C9486001201000202000010010003002F
:1000800000010102030104030904140342006C008F
:10009000750062006200460069007300680000009D
:1000A00020034800610063006B00650072002D00B2
:1000B0004A0065006F007000610072006400790002
:1000C00000000E03300030003000300030003000FF
:1000D000000011241FBECFEFD4E0DEBFCDBF11E082
:1000E000A0E0B1E0E6EFF7E102C005900D92A23F7B
:1000F000B107D9F722E0A2EFB1E001C01D92A6300E
:10010000B207E1F70E9444020C94F90B0C94000032
:1001100095B19F7195B995B18295880F807E982B86
:1001200095B9089584B1806E84B90895CF93C82F8E
:100130008A3019F48DE00E949600E8ECF0E090819E
:1001400095FFFDCFC093CE0080E090E0CF91089561
:1001500086E08093CA00E9ECF0E0808188608083CB
:1001600087E68093CC0080E091E090930302809337
:10017000020208950E94920086E090E00E948800AA
:1001800087E090E00E9488000E94A80086E090E04E
:100190000E9488000E949F0278942EE031E049E09E
:1001A00050E061E070E08FE691E00E94A0080895C1
:1001B0000895089508950F931F93CF93DF93CDB7BC
:1001C000DEB7C854D1090FB6F894DEBF0FBECDBF5D
:1001D000833009F04DC140E2BE016F5F7F4F0E9446
:1001E0009C0319A28981883669F030F48F3351F06D
:1001F000833609F01BC11AC0893671F0803709F0C7
:1002000015C11EC08AE1E9E7F1E0DE019196019097
:100210000D928A95E1F713C184E1E3E9F1E0DE0193
:10022000919601900D928A95E1F709C18BE1E7EA79
:10023000F1E0DE01919601900D928A95E1F7FFC001
:100240008E010F5D1F4F80E790E7A0E7B0E089A324
:100250009AA3ABA3BCA36091F5017091F6018091C4
:10026000F7019091F8012AE030E0A8010E945A08B5
:10027000F80101900020E9F731978AE390E091833B
:1002800080834AE050E0BE016F5B7F4F8091FB01AD
:1002900090E00E943908BE016F5B7F4FC8010E9449
:1002A0002E088091FA01823009F128F4882341F068
:1002B0008130E9F510C0833021F18430C1F52CC0C4
:1002C000FE01B19601900020E9F731978EE490E0AD
:1002D0009183808336C0FE01B19601900020E9F73A
:1002E00031978FE490E0918380832BC0FE01B1961B
:1002F00001900020E9F7319785E490E091838083B5
:1003000020C0FE01B19601900020E9F731978DE4FD
:1003100090E09183808315C0FE01B196019000208A
:10032000E9F7319783E590E0918380830AC0FE016D
:10033000B19601900020E9F731978FE390E0918327
:1003400080838091F901813079F018F0823031F5A5
:100350001AC0FE01B19601900020E9F7319781E3C0
:1003600090E09183808324C0FE01B196019000202B
:10037000E9F7319781E39EE2A5E3B0E080839183C2
:10038000A283B38315C0FE01B19601900020E9F766
:10039000319782E390E0918380830AC0FE01B19699
:1003A00001900020E9F731978FE390E091838083FB
:1003B0008E010F5D1F4FD8010D900020E9F71197B6
:1003C00086E0E2ECF1E001900D928A95E1F78091F0
:1003D000F4014AE050E0BE016F5B7F4F869590E0EC
:1003E0000E943908BE016F5B7F4FC8010E942E0832
:1003F000D8010D900020E9F7119786E0E8ECF1E0D4
:1004000001900D928A95E1F78091F4014AE050E065
:10041000BE016F5B7F4F817090E00E943908BE0182
:100420006F5B7F4FC8010E942E0809C080E1EEEC8F
:10043000F1E0DE01919601900D928A95E1F7BE01FF
:100440006F5D7F4FFB0101900020E9F731978DE050
:100450009AE0A0E080839183A283FB0101900020B9
:10046000E9F73197AF01461B570B84E00E94B203B6
:10047000C85BDF4F0FB6F894DEBF0FBECDBFDF9174
:10048000CF911F910F910895CF93DF93CDB7DEB732
:10049000A0970FB6F894DEBF0FBECDBF0E94BA0082
:1004A00082E090E00E948800912C0F2EFEEDAF2E8E
:1004B000F1E0BF2EF02D0F2EFEE0CF2EF1E0DF2E6B
:1004C000F02D0F2EF7EEEF2EF1E0FF2EF02D8E0126
:1004D0000F5F1F4F86E090E00E94880093941F9268
:1004E0009F92BF92AF92DF92CF920E948E081982A4
:1004F0001F929F92FF92EF921F930F930E94D10839
:10050000F80101900020E9F73197AF01401B510B32
:10051000B80184E00E94B20382E090E00E9488006B
:100520002FEF81EE94E0215080409040E1F700C031
:1005300000000FB6F894DEBF0FBECDBFCBCF80EA70
:100540008093D80086E089BD09B400FEFDCF80E825
:100550008093D8001092E0001092F2018FEF809308
:1005600025013C9888E08093E20008952F923F9205
:100570004F925F927F928F929F92AF92CF92DF9233
:10058000EF92FF920F931F93CF93DF93ECE2F1E092
:100590008EE291E041E00F2EF9EECF2ED12CF02D1E
:1005A0000F2EFBEEEF2EF12CF02DAA24A3940CEECF
:1005B00010E06DEE70E00F2EF0EF4F2E512CF02D6D
:1005C0006894992492F8812C6894772474F8DF0158
:1005D00020812F3F59F1E6014883E701A88220815D
:1005E000E80128831C019C0121503109E90128817F
:1005F000203841F0203441F0203241F0203141F4E4
:10060000372D07C030E405C030E303C030E201C03D
:10061000382DE1012881232BEB0128832C9120FF29
:1006200003C0D2011C9202C0E20198824F5F34964F
:100630000496453061F6EAEEF0E08EE180831082A8
:10064000DF91CF911F910F91FF90EF90DF90CF90AE
:10065000AF909F908F907F905F904F903F902F90A2
:100660000895E8EEF0E080818570E9F30895E8EE02
:10067000F0E0808182FFFDCF08958F929F92AF922C
:10068000BF92CF92DF92EF92FF920F931F93CF937F
:10069000DF93D82EE42FF0E02E173F0710F4C22E80
:1006A00001C0C42E062F172F6894992494F80F2E9A
:1006B000F8EEEF2EF12CF02D0F2EFEEFBF2EF02DC9
:1006C000C1EFD0E0A12C01C08A2C0E94310382FC32
:1006D00026C02C2D80E18C1508F4292D2223D9F079
:1006E000F801922FDD2011F0808101C08491888370
:1006F000915031969111F6CF622F615070E06F5F8B
:100700007F4F060F171FC21AF701B082C110DCCF4E
:100710002031D1F204C0F701B082C110D5CFDF91F2
:10072000CF911F910F91FF90EF90DF90CF90BF90EE
:10073000AF909F908F9008958093E9009091F20080
:10074000842F941708F4892F882359F0262FE62F39
:10075000F72FA1EFB0E09C9191939E2F921B9817D9
:10076000D0F30895CF93DF93442329F18093E900D8
:10077000E8EEF0E0808180FFFDCF8091F2008111F2
:100780001CC0962FE62FF72FA8EEB0E0C1EFD0E007
:100790008C9185FF02C08081888331968E2F891BC2
:1007A0008417B0F3E8EEF0E080818E7F80838FE7DE
:1007B000808381E003C080E001C080E0DF91CF91C1
:1007C00008951F920F920FB60F9211248F93EF93FB
:1007D000FF93E1EEF0E08081108283FF12C010925F
:1007E000E90081E08093EB001092EC0082E18093BD
:1007F000ED0088E08093F0001092F2018FEF80937B
:100800002501FF91EF918F910F900FBE0F901F90D8
:1008100018951F920F920FB60F9211242F923F92AC
:100820004F925F926F927F928F929F92AF92BF9200
:10083000CF92DF92EF92FF920F931F932F933F93EC
:100840004F935F936F937F938F939F93AF93BF93D8
:10085000EF93FF93CF93DF93CDB7DEB72997DEBF3A
:10086000CDBF8091F40080FF8FC21092E90080918B
:10087000E80083FF58C2E1EFF0E050814081208121
:100880003081932F80E0822B608170813081E08104
:1008900022EF2093E800463009F05AC11E2F00E0F5
:1008A000032B811523E0920709F42AC148F481152E
:1008B00041E09407F9F08115924009F045C10CC060
:1008C0008230A3E09A0709F42DC108F422C18330D5
:1008D000934009F039C12FC12CE331E03D832C83D3
:1008E0006CE571E0A0E040E050E0FF24F394E12CDF
:1008F00069011BC0E4E7F0E044919801BF0180E08A
:100900000E943D034AC2F901E80FF91FBF2DE081A3
:10091000EF3F09F4BE2DAB0F04968031910599F796
:10092000205F3F4F2617370711F0CA01ECCFDD8259
:10093000CC828A2F880F880F880F8A1B825D89835B
:1009400090E00E94F606E82EF92E89E0D7018C93FC
:1009500082E011968C931197E9811296EC9312978D
:1009600013961C92139714968C93149781E0159606
:100970008C93159716961C92169780E817968C9371
:1009800017978AEF18968C93189719960F2EF2E204
:10099000AF2EF1E0BF2EF02D0F2EFFE18F2EF1E0F4
:1009A0009F2EF02D0F2EFCE16F2EF1E07F2EF02D0B
:1009B00040E050E0412C512C312CDD24D394232CE9
:1009C0008FE691E01B830A83FD0188C0D801A20F46
:1009D000B31F6D2DAC91AF3F09F4622DC60E2C5F95
:1009E0003F4F2031310591F71D830C8319E01083AF
:1009F00024E0218372831382C4829A01D5016D9110
:100A00005D016583D4016D914D016683D3016D91C4
:100A10003D016783108671110CC0BF013996ACE5AA
:100A2000B1E01D911193A817B907D9F7FB017C9686
:100A300001C03996CC2009F446C022953295307F0A
:100A40003227207F3227215C3E4F11E059874887AB
:100A50006C817D813F832E83A90143505109DA01C6
:100A60000C910F3F39F1B7E0B08345E04183402F4F
:100A7000479544274795412B4283013441F0003488
:100A800041F0013841F0003841F442E007C04D2DFB
:100A900005C04D2D03C042E001C043E04383AE8159
:100AA000BF8112974C9144831582AE81BF814C91D6
:100AB000468337961F5F2C5F3F4F153059F64885A8
:100AC00059857D836C834F5F5F4F0C811D81005F73
:100AD0001F4F1D830C834230510531F0742F92015A
:100AE000C32C0C811D8172CF0A811B819801498121
:100AF000B70181E00E943D03C7010E9491074DC1EB
:100B0000E6E8F0E044919801BF0180E00E943D03D7
:100B100044C1EAE8F0E044919801BF0180E00E94FE
:100B20003D033BC1E0EAF0E044919801BF0180E061
:100B30000E943D0332C1E2ECF0E044919801BF0114
:100B400080E00E943D0329C181E28093EB0025C132
:100B5000453061F42EEF2093E800E8EEF0E02081CC
:100B600020FFFDCF80688093E30017C1372F20E07E
:100B7000262B493099F451113EC0019759F481E078
:100B80008093F2018EEF8093E800109225010E947D
:100B9000B60203C181E28093EB00FFC0483081F4CC
:100BA000503809F043C0E8EEF0E0808180FFFDCFCF
:100BB0008091F2018093F1008EEF8093E800EDC008
:100BC0004132C9F4513A09F043C0E8EEF0E08081C7
:100BD00080FFFDCF0E94D800E5EFF1E08CEF91E0BF
:100BE000A1EFB0E021912C93E817F907D9F78EEF28
:100BF0008093E800D2C04032C9F4513209F059C0A4
:100C00000E943703E5EFF1E08CEF91E0A1EFB0E057
:100C10002C912193E817F907D9F7E8EEF0E08BEF74
:100C200080838EEF80830E94D900B7C0423281F466
:100C3000513209F04FC08093F401E8EEF0E080817A
:100C400080FFFDCF8EEF8093E8000E94DA00A5C000
:100C500041111AC0E8EEF0E0808180FFFDCF5238EC
:100C600051F4E9EEF0E020838091EB0085FB8827CA
:100C700080F9108201C080E0E1EFF0E08083108213
:100C80008EEF8093E80089C04B3099F4503211F018
:100C9000511149C02230310540F4209325018EEFD7
:100CA0008093E8000E94B60278C081E28093EB0056
:100CB00074C04A3079F45038B1F5E8EEF0E0808144
:100CC00080FFFDCF809125018093F1008EEF80930E
:100CD000E80063C0413011F0433029F5523019F576
:100CE000892B09F52F773327922F91509430D8F420
:100CF0009EEF9093E8002093E900433021F481E2D5
:100D00008093EB004AC089E18093EB0081E090E0A2
:100D1000AC0102C0440F551F2A95E2F7EAEEF0E05D
:100D2000408310823AC081E28093EB002DC0122FE5
:100D3000808190E0022E02C0959587950A94E2F793
:100D400080FF19C0DA012C93DB018C9182FF13C064
:100D50008091F200882341F06091F20070E0822FD0
:100D60000E94DB001093E900E8EEF0E089EF808359
:100D70008FE7808312C02F5F3F4F25303105B9F6D2
:100D800081E28093EB0009C021E030E0E4EFF0E085
:100D900049EE50E068EE70E0CACF29960FB6F8949D
:100DA000DEBF0FBECDBFDF91CF91FF91EF91BF911D
:100DB000AF919F918F917F916F915F914F913F91F3
:100DC0002F911F910F91FF90EF90DF90CF90BF90E8
:100DD000AF909F908F907F906F905F904F903F90DB
:100DE0002F900F900FBE0F901F9018950F931F9389
:100DF000CF93DF938230910510F482E090E0E09190
:100E0000FE01F091FF0120E030E0C0E0D0E023C01F
:100E10004081518148175907A8F04817590761F4D4
:100E200082819381209719F09B838A832EC09093AF
:100E3000FF018093FE0129C02115310529F04217D9
:100E4000530710F0A90102C0BE01DF010281138126
:100E5000EF019A01F8013097D9F62115310509F112
:100E6000281B390B2430310590F412968D919C91FA
:100E700013976115710521F0FB019383828304C0F0
:100E80009093FF018093FE01FD01329644C0FD0165
:100E9000E20FF31F81939193225031092D933C93DC
:100EA0003AC02091FC013091FD01232B41F42091A7
:100EB0002801309129013093FD012093FC012091FC
:100EC0002601309127012115310541F42DB73EB798
:100ED00040912A0150912B01241B350BE091FC011C
:100EE000F091FD01E217F307A0F42E1B3F0B28172A
:100EF000390778F0AC014E5F5F4F2417350748F093
:100F00004E0F5F1F5093FD014093FC01819391931D
:100F100002C0E0E0F0E0CF01DF91CF911F910F918F
:100F20000895EF92FF920F931F93CF93DF93009753
:100F300009F48FC0DC01129713961C921E9212972F
:100F4000E090FE01F090FF01E114F10489F42D918D
:100F50003C911197280F391F8091FC019091FD0160
:100F60008217930789F5B093FD01A093FC0171C02E
:100F7000E70120E030E001C0EA01CA17DB0738F4DE
:100F80004A815B819E0141155105B1F722C0BC0128
:100F900062507109FB01D383C28300811181AC01CE
:100FA000400F511F4C175D0761F448815981400F74
:100FB000511F4E5F5F4F518340834A815B81538352
:100FC00042832115310529F4B093FF01A093FE015E
:100FD00040C0F901B383A283E90169917991C60FF9
:100FE000D71FAC17BD0779F4DC015E914E91460F17
:100FF000571F4E5F5F4F5183408312968D919C9196
:10100000139793838283A0E0B0E002C0D7017C01F4
:10101000F701828193810097C9F7C7010296208169
:101020003181820F931F2091FC013091FD0128171F
:10103000390779F4109729F41092FF011092FE01FC
:1010400004C013961C921E921297F092FD01E0923A
:10105000FC01CDB7DEB7E6E00C94EA0BFB01DC0146
:101060000D900020E9F7119701900D920020E1F713
:101070000895FB019F01E8944230C4F04532B4F476
:101080004A3029F497FB1EF4909581959F4F642F69
:1010900077270E948C0B805D8A330CF0895D8193E9
:1010A000CB010097A1F716F45DE251931082C901BC
:1010B0000C94E70AFA01CF93FF93EF93223044F1A7
:1010C000253234F5C22FE894CA3049F497FB3EF438
:1010D00090958095709561957F4F8F4F9F4F2C2FE6
:1010E000332744275527FF93EF930E94A00BEF91DE
:1010F000FF91605D6A330CF0695D6193B901CA01CB
:10110000605070408040904051F716F4CDE2C1939A
:1011100010828F919F91CF910C94E70AA0E0B0E0EC
:10112000E4E9F8E00C94D20BCE010996AC016F8192
:1011300078858D819E810E94F308E2E00C94EE0B8D
:10114000A0E0B0E0E6EAF8E00C94C80B6B014A01BD
:101150007901D90113962C9121FF1BC08C01C0E0AD
:10116000D0E010C0D7011896ED91FC911997B70106
:10117000D8018D918D010995892B69F40A151B05FC
:1011800089F72196C815D90531F05801AC0CBD1C62
:10119000F5CFC0E0D0E0CE01CDB7DEB7ECE00C94E7
:1011A000E40BAEE0B0E0E7EDF8E00C94D00B0D8975
:1011B0001E8986E08C831A8309838FEF9FE79E83C5
:1011C0008D83CE014996AC016F89788DCE01019651
:1011D0000E94F308EF81F885E00FF11F10822E9630
:1011E000E4E00C94EC0BACE0B0E0E9EFF8E00C9438
:1011F000C20B7C016B018A01FC011782168283817C
:1012000081FFC8C188248394912C8C0E9D1EF70108
:101210009381F60193FD859193FF81916F0188235E
:1012200009F4B4C1853239F493FD859193FF81911E
:101230006F01853229F4B70190E00E94F70AE7CFE9
:10124000512C312C20E02032A8F48B3261F028F4AC
:10125000803251F0833271F40BC08D3239F080331B
:1012600049F421602AC02260246027C0286025C07C
:10127000206123C027FD29C0382F30533A3088F42D
:1012800026FF07C0852D6AE00E94830B582E530E5F
:1012900014C0832D6AE00E94830B382E330E206227
:1012A0000CC08E3221F426FD71C1206406C08C363C
:1012B00011F4206802C0883641F4F60193FD85914F
:1012C00093FF81916F018111BECF982F9554933078
:1012D00018F09052933028F40C5F1F4FFFE3F9830E
:1012E0000DC0833631F0833771F0833509F05EC06D
:1012F00023C0F801808189830E5F1F4F44244394EB
:10130000512C540115C03801F2E06F0E711CF80128
:10131000A080B18026FF03C0652D70E002C06FEF92
:101320007FEFC5012C870E94DC0A2C0183012C85EC
:101330006FE7262E222218C03801F2E06F0E711CD2
:10134000F801A080B18026FF03C0652D70E002C0C7
:101350006FEF7FEFC5012C870E94D10A2C012C85ED
:1013600050E8252E222A830123FC1CC006C0B701A9
:1013700080E290E00E94F70A3A94832D90E04816AC
:101380005906A8F30FC0F50127FC859127FE81912E
:101390005F01B70190E00E94F70A31103A94F1E042
:1013A0004F1A51084114510471F7EDC0843611F001
:1013B000893641F5F80127FF07C06081718182817C
:1013C00093810C5F1F4F08C060817181882777FD72
:1013D0008095982F0E5F1F4F4FE6B42EB22297FFD5
:1013E00009C090958095709561957F4F8F4F9F4F65
:1013F000F0E8BF2A2AE030E0A4010E94230BA82EC7
:10140000A81843C0853731F43FEEB32EB2222AE04C
:1014100030E024C099EFB92EB2228F36B9F020F413
:10142000883509F0B3C00DC0803721F0883709F046
:10143000ADC002C020E1B22AB4FE0BC084E0B82ADD
:1014400008C024FF09C0E6E0BE2A06C028E030E05C
:1014500005C020E130E002C020E132E0F801B7FE33
:1014600007C060817181828193810C5F1F4F06C02C
:101470006081718180E090E00E5F1F4FA4010E94A7
:10148000230BA82EA818FFE7BF22B6FE0BC02B2DFA
:101490002E7FA51450F4B4FE0AC0B2FC08C02B2D58
:1014A0002E7E05C07A2C2B2D03C07A2C01C0752C02
:1014B00024FF0DC0FE01EA0DF11D8081803311F47F
:1014C000297E09C022FF06C07394739404C0822F42
:1014D000867809F0739423FD14C020FF0FC05A2CA6
:1014E000731460F4530C5718732C08C0B70180E2D2
:1014F00090E02C870E94F70A73942C857314B0F344
:1015000004C0731410F4371801C0312C24FF12C02A
:10151000B70180E390E02C870E94F70A2C8522FF18
:101520001EC021FF03C088E590E002C088E790E07C
:10153000B7010CC0822F867891F021FD02C080E2B5
:1015400001C08BE227FD8DE2B70190E00E94F70A0F
:1015500006C0B70180E390E00E94F70A5A94A514F0
:10156000C0F3AA94F401EA0DF11DB701808190E067
:101570000E94F70AA110F5CF06C0B70180E290E003
:101580000E94F70A3A943110F8CF41CEF701268134
:10159000378102C02FEF3FEFC9012C96E2E10C9496
:1015A000DE0BFC010590615070400110D8F780956A
:1015B00090958E0F9F1F0895FC016150704001901F
:1015C0000110D8F7809590958E0F9F1F0895DC012C
:1015D000FC01672F71917723E1F7329704C07C916A
:1015E0006D9370836291AE17BF07C8F308950F9390
:1015F0001F93CF93DF938C01EB018B8181FD03C09F
:101600000FEF1FEF1AC082FF0DC02E813F818C812A
:101610009D812817390764F4E881F9810193F983E2
:10162000E88306C0E885F985802F0995892B41F765
:101630008E819F8101969F838E83C801DF91CF9118
:101640001F910F910895FA01AA27283061F12031E6
:1016500091F1E8946F936E7F6E5F7F4F8F4F9F4F36
:10166000AF4FB1E040D0B4E03ED0670F781F891F84
:101670009A1FA11D680F791F8A1F911DA11D6A0F56
:10168000711D811D911DA11D22D009F468943F9107
:10169000062E000C3019000C000C3019305D31930F
:1016A000CEF6CF010895462F4770405D4193B3E0D9
:1016B0000FD0C9F7F6CF462F4F70405D4A3318F070
:1016C000495D31FD4052419302D0A9F7EACFB4E021
:1016D000A6959795879577956795BA95C9F70097D9
:1016E0006105710508959B01AC010A2E069457957A
:1016F000479537952795BA95C9F7620F731F841FD1
:10170000951FA01D0895002480FD060E660F11F0A0
:101710008695D1F7802D0895AA1BBB1B51E107C008
:10172000AA1FBB1FA617B70710F0A61BB70B881F71
:10173000991F5A95A9F780959095BC01CD01089500
:10174000A1E21A2EAA1BBB1BFD010DC0AA1FBB1FC5
:10175000EE1FFF1FA217B307E407F50720F0A21B37
:10176000B30BE40BF50B661F771F881F991F1A94A4
:1017700069F760957095809590959B01AC01BD01CE
:10178000CF0108952F923F924F925F926F927F9276
:101790008F929F92AF92BF92CF92DF92EF92FF9281
:1017A0000F931F93CF93DF93CDB7DEB7CA1BDB0B2D
:1017B0000FB6F894DEBF0FBECDBF09942A883988D2
:1017C00048885F846E847D848C849B84AA84B984D9
:1017D000C884DF80EE80FD800C811B81AA81B981E5
:1017E000CE0FD11D0FB6F894DEBF0FBECDBFED01F9
:0617F0000895F894FFCFFC
:1017F600000000020000000096000000000000004B
:101806000002000000009600000000000100FF0238
:1018160000FF020AFFFF000006022000FF20020070
:10182600C11002408020060081200600FF20020031
:10183600C1100240FF200600FF200600FF20020024
:10184600FF200200802006008120060005240010EB
:1018560001052401010104240206052406000149AC
:101866006E69742E2E2E2E0A0056616C69642063F2
:101876006F6D6D616E64733A203F20682069206346
:10188600207000557844494C204344432044656DFC
:101896006F2056312E300028632920323031312016
:1018A60052657573636820456C656B74726F6E69FB
:1018B6006B00205254533D00204454523D00696E43
:1018C60076616C696420636F6D6D616E640074652A
:1018D60073742025640A00746573742025640D0AE8
:0218E600000000
:00000001FF
